:100000000C9450030C947F030C947F030C947F0397
:100010000C947F030C947F030C947F030C947F0358
:100020000C947F030C947F030C947F030C947F0348
:100030000C947F030C947F030C947F030C947F0338
:100040000C947F030C947F030C947F030C947F0328
:100050000C947F030C947F030C947F030C947F0318
:100060000C947F030C94F20A0C947F030C944B0BBA
:100070000C947F030C947F030C947F030C947F03F8
:100080000C947F030C947F030C947F030C947F03E8
:100090000C94C30A0C947F030C94210B0C947F03E3
:1000A0000C947F030C947F030C947F030C947F03C8
:1000B0000C947F030C947F030C947F030C94070C27
:1000C0000C947F030C947F030C947F030C947F03A8
:1000D0000C947F030C947F030C947F030C947F0398
:1000E0000C947F030C9474060C9489060C94D1052F
:1000F0000C9405060C94C4060C947F030C946206C1
:100100000C947F030C947F030C947F030C947F0367
:100110000C947F030C947F030C947F030C949B0638
:1001200045464765666700202B2D2E30313233342B
:10013000353637383968000A7472616E736D6973C9
:1001400073696F6E206661696C65642C206D7573D0
:100150007420626520696E20504C4C5F4F4E2073B6
:10016000746174650A000A7472616E736D6974203B
:100170006572726F723A206461746120657863659C
:100180006564656420313235206279746573002EB0
:100190000A2053656520576562626F744C6962205E
:1001A0006D616E75616C206F6E2066696C654F7055
:1001B000656E20696E2046696C6553797374656D50
:1001C0002F4641542E6820666F72206D6F72652035
:1001D000696E666F2E0A00546865206D6F64652035
:1001E000706172616D6574657220697320696E76E5
:1001F000616C69640020342E204953502050726F86
:100200006772616D6D657220697320706C756767C8
:10021000656420696E0020332E205468652066696D
:100220006C6520616C7265616479206578697374AE
:10023000732062757420617320616E20696E636F34
:100240006D70617469626C6520656E636F64696E60
:10025000670A0020322E20546865207553442063BD
:10026000617264206973206E6F7420696E207468F7
:100270006520736C6F740A0020312E20546865204D
:100280006469736B2069732066756C6C0A00457233
:10029000726F722063617573656420627920616E8C
:1002A0007920636F6D62696E6174696F6E206F662D
:1002B0002074686573653A0A00596F75206172652C
:1002C00020747279696E6720746F20777269746523
:1002D00020746F20612072656164206F6E6C7920DC
:1002E00066696C6500546865206469726563746F43
:1002F000727920646F65736E2774206578697374F2
:10030000005468652066696C6520616C7265616483
:100310007920657869737473207768656E206F70D3
:10032000656E696E6720666F72207772697465000A
:100330005468652066696C6520646F65736E277408
:10034000206578697374207768656E206F70656EBC
:10035000696E6720666F722072656164000A436F80
:10036000756C646E277420637265617465206669BC
:100370006C652C206572726F723A2025640A200029
:100380000A676F696E6720696E746F205258206D1E
:100390006F64650A000A656E746572696E67207421
:1003A00072616E736D6974206D6F64650A000A0A6C
:1003B00041786F6E204D6F746520696E6974696154
:1003C0007465642E0A5472616E736D6974206F6E69
:1003D000204368616E6E656C2025642E0A0A000A4F
:1003E000525353493A25642045443A256420524EDD
:1003F000443A25640A002563000A53797374656DD5
:1004000020537461727465640A0051041051042011
:100410005104405104805704045704085704805D78
:1004200004015D04025D04045D04085D04105D04C4
:10043000205D04405D0480630401630402630404DE
:10044000630408630410630420630440630480E4CD
:100450000C2500240023002B002A0029002E002D4B
:10046000002C00310030002F00DE02006E00024739
:10047000003500024400061304E202006E00044846
:10048000003500044400040000E602016F00028809
:10049000003600028000060D04EA02016F00048AA3
:1004A000003600048000041004EE02016F00088C86
:1004B000003600088000021304F20202700002B34A
:1004C00000370002B000060000F60202700004B41B
:1004D00000370004B000040000FA02037100029823
:1004E000003800029000062804FE02037100049AFE
:1004F000003800049000042B040203037100089CE0
:10050000003800089000022E04060304720002A8BE
:1005100000390002A0000600000A0304720004AAC9
:1005200000390004A0000400000E0304720008ACAF
:1005300000390008A0000200001203057300022821
:10054000013A000220010600001603057300042A88
:10055000013A000420010400001A03057300082C6E
:10056000013A000820010200001E03460045000079
:1005700000023388440001440002450008000001E5
:1005800069046E0001350001000000000100000157
:100590000000010000290384008100FF0003FFDF49
:1005A00080000180000281000881001089046F0032
:1005B0000136000186006F002036002081004000D7
:1005C000003403B200B1000000023388B00001B073
:1005D0000002B10008000001B904700001370001F9
:1005E000000000000100000100000100003F039432
:1005F000009100FF0003FFDF9000019000029100D6
:1006000008910010D90471000138000196007100B2
:100610002038002091004034044A03A400A100FFC8
:100620000003FFDFA00001A00002A10008A100104C
:100630000905720001390001A6007200203900206E
:10064000A100400000550324012101FF0003FFDF4A
:100650002001012001022101082101103905730048
:10066000013A000126017300203A002021014000D8
:100670000055736572204572726F723A25640A00E4
:10068000576562626F744C6962204572726F723A8C
:1006900025640A00D00E860FA20F5B0F8D0F710F1D
:1006A00011241FBECFEFD1E4DEBFCDBFE4E5F0E003
:1006B00080818093A004E4E5F0E0108288E10FB629
:1006C000F89480936000109260000FBE12E0A0E0EA
:1006D000B2E0E0E9F9E200E00BBF02C007900D9242
:1006E000A63DB107D9F714E0A6EDB2E001C01D9216
:1006F000A03AB107E1F70E94B60D0C94AA130C942E
:100700000000DF93CF93CDB7DEB7EDE4F1E0808159
:10071000877F8083EEE4F1E0808181608083EEE476
:10072000F1E0808182608083EEE4F1E0808184608A
:100730008083EEE4F1E0808188608083EEE4F1E084
:10074000808180648083EEE4F1E080818061808339
:10075000E1E5F1E080818F7B8083E1E5F1E080815C
:1007600080618083E1E5F1E0809100028F70982F35
:100770009F708081807F892B8083E4E4F1E0808119
:1007800080628083E5E4F1E08081807F8083E5E41E
:10079000F1E0808180638083E5E4F1E08081806C1A
:1007A0008083ECE4F1E080818C7F8083CF91DF91C6
:1007B0000895DF93CF93CDB7DEB7E1E4F1E0808118
:1007C0008F718F31D1F3CF91DF910895DF93CF9364
:1007D000CDB7DEB70E94D903A9E3B1E0E9E3F1E0C8
:1007E00080818D7F8C930E94D903A9E3B1E0E9E376
:1007F000F1E0808181608C93E1E4F1E080818F7190
:100800008830D1F70E9481037894CF91DF910895C9
:10081000DF93CF93CDB7DEB7E2E4F1E08081807E55
:1008200088608083CF91DF910895DF93CF930F92FB
:10083000CDB7DEB789830E94D9038981813081F4E5
:10084000E1E4F1E080818F71883021F00E9408049A
:100850000E94D903E9E3F1E080818260808308C0CF
:100860008981882329F4E9E3F1E080818D7F808309
:100870000F90CF91DF910895DF93CF930F92CDB773
:10088000DEB7898389818B3018F48BE0898305C0BA
:1008900089818B3110F08AE18983E8E4F1E0898174
:1008A0008F71982F9F718081807E892B808369E171
:1008B00070E080E090E00E94630E0F90CF91DF9196
:1008C0000895DF93CF930F92CDB7DEB71982A8E4D6
:1008D000B1E0E8E4F1E0808180688C936CE870E03E
:1008E00080E090E00E94630EE8E4F1E080818F7187
:1008F000898389810F90CF91DF910895DF93CF9302
:10090000CDB7DEB70E94D903E2E4F1E08081807EBA
:10091000896080836EE670E080E090E00E94630E64
:10092000EFE4F1E0808181708823D1F7CF91DF91EE
:100930000895DF93CF93CDB7DEB70E94D903E1E4EA
:10094000F1E080818F71883069F41092DD02E2E479
:10095000F1E08081807E866080838091DD02882343
:10096000E1F30CC0E1E4F1E080818F71893031F472
:10097000E2E4F1E08081807E86608083E1E4F1E062
:1009800080818F718630D1F7CF91DF910895DF9309
:10099000CF93CDB7DEB70E94D9038FEF8093DC02EF
:1009A000E1E4F1E080818F71893069F4E2E4F1E003
:1009B0008081807E826080838091DC028823E1F7E1
:1009C0001092D90210C087E391E000D00F92EDB7EA
:1009D000FEB7319621E02083928381830E94460EE8
:1009E0000F900F900F900E94D903E2E4F1E0808114
:1009F000807E89608083CF91DF910895DF93CF93CC
:100A00000F92CDB7DEB789838091D9028F5F809333
:100A1000D902E0E8F1E08091D9028E5F8083809175
:100A2000D902882F90E080589E4FFC0189818083F5
:100A30000F90CF91DF910895DF93CF9300D0CDB782
:100A4000DEB79A83898389819A81009799F12DC0B5
:100A50008091D9028F5F8093D9028091D9028E371D
:100A600080F48091D902882F90E080589E4FDC015D
:100A7000E981FA8180818C9389819A8101969A8398
:100A800089838091D9028E3781F486E691E000D087
:100A90000F92EDB7FEB7319621E0208392838183D8
:100AA0000E94460E0F900F900F90E981FA8180818D
:100AB000882371F6E0E8F1E08091D9028E5F8083AF
:100AC0000F900F90CF91DF910895DF93CF93CDB723
:100AD000DEB7E6E4F1E080818F718093D602E6E430
:100AE000F1E08081829586958770837080931204EF
:100AF000CF91DF910895DF93CF93CDB7DEB70E94FA
:100B00007E04CF91DF910895DF93CF93CDB7DEB709
:100B10000E94C704CF91DF910895DF93CF93CDB7A3
:100B2000DEB70E949904CF91DF910895DF93CF93B0
:100B30000F92CDB7DEB789838981813019F40E9485
:100B40007E0402C00E9499040F90CF91DF91089516
:100B5000DF93CF93CDB7DEB70E940804CF91DF912A
:100B60000895DF93CF93CDB7DEB781E00E941504DF
:100B7000CF91DF910895DF93CF93CDB7DEB780E0BB
:100B80000E941504CF91DF910895DF93CF93CDB7E5
:100B9000DEB7E0E8F1E010821092D902CF91DF9148
:100BA00008951F920F920FB60F9200905B000F9264
:100BB00011242F933F934F935F936F937F938F9362
:100BC0009F93AF93BF93EF93FF93DF93CF93CDB7F3
:100BD000DEB70E946505E7E4F1E08FEF8083CF91F7
:100BE000DF91FF91EF91BF91AF919F918F917F9195
:100BF0006F915F914F913F912F910F9000925B0009
:100C00000F900FBE0F901F9018951F920F920FB666
:100C10000F9200905B000F9211242F933F938F93BC
:100C20009F93EF93FF93DF93CF9300D0CDB7DEB7C1
:100C3000E6E4F1E080818078882381F11A821982CC
:100C4000EBE7F1E080818A83198211C08981282F26
:100C500030E08981882F90E080589E4FFC01808190
:100C6000F901ED5EFB4F808389818F5F89838981E4
:100C7000282F30E08A81882F90E0029728173907C3
:100C80002CF38A81882F90E080589E4FFC01808150
:100C90008093D8028FEF8093DA0202C01092DA02BA
:100CA0000F900F90CF91DF91FF91EF919F918F91D6
:100CB0003F912F910F9000925B000F900FBE0F900D
:100CC0001F9018951F920F920FB60F921124DF9369
:100CD000CF93CDB7DEB71092DC02CF91DF910F90AA
:100CE0000FBE0F901F9018951F920F920FB60F9284
:100CF00011248F93DF93CF93CDB7DEB78FEF80931F
:100D0000DD02CF91DF918F910F900FBE0F901F905A
:100D100018951F920F920FB60F921124DF93CF9365
:100D2000CDB7DEB71092DD02CF91DF910F900FBEED
:100D30000F901F9018951F920F920FB60F92009070
:100D40005B000F9211248F93EF93FF93DF93CF9368
:100D5000CDB7DEB7E1E5F1E080818F7B80838FEF57
:100D60008093DB02E1E5F1E0808180648083CF91B4
:100D7000DF91FF91EF918F910F9000925B000F90A8
:100D80000FBE0F901F9018951F920F920FB60F92E3
:100D900000905B000F9211248F93EF93FF93DF93EA
:100DA000CF93CDB7DEB7E7E4F1E080818093D7023F
:100DB000CF91DF91FF91EF918F910F9000925B00A7
:100DC0000F900FBE0F901F901895DF93CF930F9247
:100DD000CDB7DEB789834DE553E08981282F3327CE
:100DE00027FD309500D000D00F92EDB7FEB73196B9
:100DF00081E0808352834183348323830E94460EA3
:100E00000F900F900F900F900F9089818F3F81F47A
:100E100080E393E000D00F92EDB7FEB7319621E06A
:100E20002083928381830E94460E0F900F900F9033
:100E300089818E3F81F481E093E000D00F92EDB77D
:100E4000FEB7319621E02083928381830E94460E73
:100E50000F900F900F9089818D3F81F485EE92E085
:100E600000D00F92EDB7FEB7319621E02083928338
:100E700081830E94460E0F900F900F9089818C3FC6
:100E800081F489EB92E000D00F92EDB7FEB7319676
:100E900021E02083928381830E94460E0F900F9061
:100EA0000F9089818B3F09F050C02EE832E000D0CE
:100EB0000F92EDB7FEB7319681E0808332832183B4
:100EC0000E94460E0F900F900F9028E732E000D05E
:100ED0000F92EDB7FEB7319681E080833283218394
:100EE0000E94460E0F900F900F9023E532E000D045
:100EF0000F92EDB7FEB7319681E080833283218374
:100F00000E94460E0F900F900F9026E132E000D025
:100F10000F92EDB7FEB7319681E080833283218353
:100F20000E94460E0F900F900F9025EF31E000D0F9
:100F30000F92EDB7FEB7319681E080833283218333
:100F40000E94460E0F900F900F9089818A3F81F486
:100F500087ED91E000D00F92EDB7FEB7319621E01A
:100F60002083928381830E94460E0F900F900F90F2
:100F7000898188232CF48BE792E00E94D80704C073
:100F80008BE792E00E94E9078FE891E000D00F9292
:100F9000EDB7FEB7319621E02083928381830E94D2
:100FA000460E0F900F900F900F90CF91DF91089504
:100FB000DF93CF9300D0CDB7DEB79A838983898141
:100FC0009A816FEF0E94940D0F900F90CF91DF9157
:100FD0000895DF93CF9300D0CDB7DEB79A8389838E
:100FE00089819A8160E00E94940D0F900F90CF91BB
:100FF000DF910895DF93CF930F92CDB7DEB789834A
:1010000089810E947F0B0F90CF91DF910895DF932C
:10101000CF93CDB7DEB70E942A0ACF91DF91089512
:101020000F931F93DF93CF9300D000D0CDB7DEB7DF
:1010300069837A838B839C8364E670E080E090E030
:101040000E94930864E670E080E090E00E949308BC
:101050000E94E603809101020E943C040EEA13E024
:101060000E946104282F30E000D000D00F92EDB72D
:10107000FEB7319681E0808312830183348323831A
:101080000E94460E0F900F900F900F900F9080E8E7
:1010900092E00E94AC088823C9F087E994E00E949E
:1010A000D80725E933E000D00F92EDB7FEB73196AF
:1010B00081E08083328321830E94460E0F900F903F
:1010C0000F900E947B0581E0809311048EE792E0EF
:1010D0000E94AC088823C1F08BE792E00E94D807F9
:1010E00020E833E000D00F92EDB7FEB7319681E0F3
:1010F0008083328321830E94460E0F900F900F90C1
:101100000E948D051092110480E090E0A0E0B0E014
:10111000BC01CD010F900F900F900F90CF91DF91F8
:101120001F910F910895DF93CF9300D000D0CDB7DA
:10113000DEB769837A838B839C8389819A81AB81B3
:10114000BC81BC01CD010E946A0C0F900F900F90E2
:101150000F90CF91DF910895DF93CF9300D00F923E
:10116000CDB7DEB79A838983E981FA818081918145
:101170000E94F80C1B82882311F481E08B838B8101
:101180000F900F900F90CF91DF910895DF93CF9341
:10119000CDB7DEB72B970FB6F894DEBF0FBECDBF2D
:1011A0006C837D838E839F83288739874A875B87FB
:1011B00082E892E00E94AC08882341F08BE792E03D
:1011C0000E94E90787E994E00E94E90782E892E03B
:1011D0000E94D109882341F08BE792E00E94D80752
:1011E00087E994E00E94D8078AE394E00E94700D9A
:1011F0008DE394E00E94700D80E494E00E94700DF5
:1012000083E494E00E94700D86E494E00E94700DE7
:1012100089E494E00E94700D8CE494E00E94700DCB
:101220008EE294E00E94700D8BE294E00E94700DBB
:1012300088E294E00E94700D83E194E00E94700DBA
:1012400080E194E00E94700D8DE094E00E94700DAA
:101250008AE094E00E94700D8AEF97E00E94200ED1
:101260009B838A8329EF33E000D00F92EDB7FEB75E
:10127000319681E08083328321830E94460E0F9055
:101280000F900F908A819B810E94200E8091110403
:10129000813031F482E092E00E941C050E948405B6
:1012A00080911104882309F06DC08091DA028823AF
:1012B000B1F181E00E949605198221C046EF53E00A
:1012C0008981882F90E0FC01ED5EFB4F8081282F03
:1012D00030E000D000D00F92EDB7FEB7319681E03C
:1012E000808352834183348323830E94460E0F9070
:1012F0000F900F900F900F9089818F5F8983898164
:10130000282F30E080911404882F90E0029728174E
:101310003907A4F20E94C50580E00E949605AFED52
:10132000B3E08091D602282F30E08091D702482F79
:1013300050E080911204682F70E08DB79EB7099736
:101340000FB6F8949EBF0FBE8DBFEDB7FEB73196B6
:1013500081E08083B283A1833483238356834583D2
:10136000708767830E94460E8DB79EB709960FB6A9
:10137000F8949EBF0FBE8DBF1092DA021092D70272
:101380001092D60280E492E4AFE0B0E0BC01CD015F
:101390002B960FB6F894DEBF0FBECDBFCF91DF9175
:1013A0000895DF93CF9300D0CDB7DEB79A838983BA
:1013B000E981FA81808191810E94F80C0F900F9051
:1013C000CF91DF910895E5E4F6E0A591B49184E032
:1013D0001A968C931A97E1E2F1E08081886080830D
:1013E00080E09AEF909329018093280188E090E0B3
:1013F0008D939C938081826080830895FB01048497
:10140000F585E02D309719F42FEF3FEF02C00995D5
:101410009C01C9010895DC011C96ED91FC911D977A
:10142000309719F42FEF3FEF02C009959C01C901D5
:1014300008958CE194E090939804809397048091B0
:1014400099048C7F8093990487E994E06FEF0E9460
:10145000940D08958AE394E060E00E94490D8DE3C5
:1014600094E060E00E94490D80E494E060E00E9416
:10147000490D83E494E060E00E94490D86E494E025
:1014800060E00E94490D89E494E060E00E94490D0B
:101490008CE494E060E00E94490D8EE294E060E00C
:1014A0000E94490D8BE294E060E00E94490D88E2C1
:1014B00094E060E00E94490D83E194E060E00E94C6
:1014C000490D80E194E060E00E94490D8DE094E0D8
:1014D00060E00E94490D8AE094E060E00E94490DBE
:1014E00089E492E040E054E863E070E00E948A0EF4
:1014F00008950F931F9380917E0290917F026FEF6A
:101500000E94220D80918002909181026FEF0E94D3
:10151000220D06E81BE0C8010E949A0C84E892E0C4
:1015200090939F0480939E041093910200939002E5
:10153000C8010E94200E82E992E090939D0480935E
:101540009C0410939F0200939E0280EA92E0909385
:101550009B0480939A048AE79BE09093AD0280936A
:10156000AC0288E192E040E052EC61E070E00E9461
:101570008A0E80918202909183026FEF0E94220D69
:101580001F910F9108951F920F920FB60F920BB6F5
:101590000F9211242F933F934F935F936F937F93F9
:1015A0008F939F93AF93BF93EF93FF93E091750257
:1015B000F0917602608189E492E00E94BE0FFF9173
:1015C000EF91BF91AF919F918F917F916F915F91BB
:1015D0004F913F912F910F900BBE0F900FBE0F9028
:1015E0001F9018951F920F920FB60F920BB60F9285
:1015F00011242F933F934F935F936F937F938F9318
:101600009F93AF93BF93EF93FF93E0914402F091C8
:101610004502608188E192E00E94BE0FFF91EF9148
:10162000BF91AF919F918F917F916F915F914F91FA
:101630003F912F910F900BBE0F900FBE0F901F90F8
:1016400018951F920F920FB60F920BB60F9211249E
:101650002F933F934F935F936F937F938F939F93BA
:10166000AF93BF93EF93FF9389E492E00E949510AC
:10167000FF91EF91BF91AF919F918F917F916F916A
:101680005F914F913F912F910F900BBE0F900FBE26
:101690000F901F9018951F920F920FB60F920BB6D6
:1016A0000F9211242F933F934F935F936F937F93E8
:1016B0008F939F93AF93BF93EF93FF9388E192E053
:1016C0000E949510FF91EF91BF91AF919F918F91E3
:1016D0007F916F915F914F913F912F910F900BBE32
:1016E0000F900FBE0F901F90189589E492E00E9412
:1016F000D80F089588E192E00E94D80F0895682FCE
:1017000089E492E00E948B1090E00895682F88E1B0
:1017100092E00E948B1090E00895FC016FB7F8945E
:1017200080912401909125012091000430910104C1
:1017300040910204509103042083318342835383F8
:1017400020912401309125013583248328173907FE
:1017500010F0D19B12C080819181A281B381805011
:101760009348AF4FBF4F80839183A283B38380910F
:10177000240190912501958384836FBF0895EF9292
:10178000FF920F931F93FC01E080F180028113818F
:101790006481758180E090E020E03DE740E050E02A
:1017A0000E94711420E03AEF40E050E00E94A4143F
:1017B0002E0D3F1D401F511FB901CA011F910F91EE
:1017C000FF90EF9008950F931F93DF93CF9300D076
:1017D00000D000D0CDB7DEB78E010F5F1F4FC8011C
:1017E0000E948D0BC8010E94BF0B26960FB6F8947D
:1017F000DEBF0FBECDBFCF91DF911F910F91089536
:10180000D19AE3E7F0E080818260808308951F929F
:101810000F920FB60F9211242F938F939F93AF9334
:10182000BF938091000490910104A0910204B091B3
:10183000030480509348AF4FBF4F809300049093B0
:101840000104A0930204B093030420919204222384
:10185000B9F1579B35C080910404882319F0815059
:101860008093040480910404882351F580919304AB
:10187000882359F4822F992787FD909597FF03C0FD
:10188000909581959F4F8093930427FD02C09FE020
:1018900001C097E020919404222341F080919304A9
:1018A000815080939304882309F49EE3109294045A
:1018B000222319F481E080939404909304044F9AB6
:1018C000BF91AF919F918F912F910F900FBE0F906D
:1018D0001F90189528EE33E040E050E00E9471140C
:1018E0000E94730C0895AF92BF92CF92DF92EF9255
:1018F000FF920F931F935B016C010E94E30B7B012E
:101900008C0101C000000E94E30B6E197F09800B5F
:10191000910B6A157B058C059D05A0F31F910F9116
:10192000FF90EF90DF90CF90BF90AF90089580919F
:1019300092040895909396048093950408951F93BC
:10194000182F80919204882309F050C010939204BC
:101950008091970490919804009749F00E940D0D92
:10196000882329F087E994E060E00E94940D80913B
:101970009E0490919F040097C9F1212F332727FDE2
:10198000309517FF17C000D000D000D0EDB7FEB7DC
:101990003196ADB7BEB712969C938E93119780E89F
:1019A00096E09383828388279927821B930B9583E4
:1019B000848312C000D000D000D0EDB7FEB73196BE
:1019C000ADB7BEB712969C938E93119781E796E0C0
:1019D00093838283358324830E94B8138DB79EB787
:1019E00006960FB6F8949EBF0FBE8DBF1F91089547
:1019F0009C01009781F0FC01859194910496FC0173
:101A0000A591B4912E5F3F4FF90194918C91892358
:101A100011F08FEF089580E008959C01009781F008
:101A2000FC01859194910296FC01A591B4912E5FE1
:101A30003F4FF90194918C91892311F08FEF089514
:101A400080E00895CF93DF939C010097F9F0FC01AB
:101A500045915491CA010296FC01A591B491FA01F5
:101A6000C591D4912E5F3F4FF90194913FB7F894FF
:101A70008C91292F209582238C93662319F08881DD
:101A8000892B02C08881822388833FBFDF91CF9159
:101A90000895CF93DF939C010097F9F0FC014591E5
:101AA0005491CA010296FC01C591D491FA01A59105
:101AB000B4912E5F3F4FF90124913FB7F89466230C
:101AC00019F08C91822B04C08C91922F90958923D0
:101AD0008C938881822B88833FBFDF91CF910895BB
:101AE000CF93DF939C010097E1F0FC0185919491E5
:101AF000FC01A591B4910296FC01C591D4912E5F91
:101B00003F4FF90124918881822341F09FB7F894D7
:101B10008C9182278C939FBF000003C087EF0E94A7
:101B20009F0CDF91CF9108951F93CF93DF93EC012A
:101B3000162F888199810097A9F03A8130FD05C060
:101B400020E0662309F421E0122F31FD06C0612F49
:101B50000E94490D8A8182608A8388819981612FE0
:101B60000E94D511DF91CF911F9108950E94190A0B
:101B70000E94E3090E94000C78940E94790A0E9456
:101B800007080E94E30B6093090470930A04809392
:101B90000B0490930C040E94100860930D04709342
:101BA0000E0480930F049093100478940E94CA113D
:101BB00080910D0490910E04A0910F04B091100437
:101BC0000097A105B10519F416C00E94CA116091D1
:101BD000090470910A0480910B0490910C042091E7
:101BE0000D0430910E0440910F04509110040E9496
:101BF0007F11882351F30E94E30B9B01AC0160939A
:101C0000090470930A0480930B0490930C04609170
:101C100005047091060480910704909108046F5F99
:101C20007F4F8F4F9F4F60930504709306048093FE
:101C30000704909308040E94C608AFCF90E008956F
:101C40004FB7F8942091C6023091C7029093C70213
:101C50008093C6024FBFC90108951F93182F8A3081
:101C600031F4E091C602F091C7028DE00995E09150
:101C7000C602F091C702812F09951F9108958AE04D
:101C80000E942D0E08958FEF9FEF0895DF93CF935D
:101C9000CDB7DEB76E817F819E01285F3F4F8D817A
:101CA000813031F488EC92E0A9010E94021405C051
:101CB00088EC92E0A9010E946A12CF91DF91089509
:101CC0000E942D0E0895653671058105910518F065
:101CD0000E94730C0895209114023091150240E087
:101CE00050E00E94711428EE33E040E050E00E9482
:101CF000A414CA01B9010E94DD110895DC011996EE
:101D00008D919C911A97FC0125913491CD01F90197
:101D100009950895DF92EF92FF920F931F93CF934F
:101D2000DF93EC017A018B01DFB6F8942D853E85B7
:101D30008F8598892817390711F080E001C08FEF4F
:101D40008D8B882381F02D853E858F859889281776
:101D5000390721F0C90160E00E94220D8F85988922
:101D60006FEF0E94220D88858160888788858B7F30
:101D7000888788858D7F888789859A850496FC0168
:101D800025913491CE01B801A701F9010995DFBE73
:101D9000DF91CF911F910F91FF90EF90DF90089509
:101DA000BF92CF92DF92EF92FF920F931F93CF9348
:101DB000DF937A018B01EC01BFB6F8944F3F8FEFB0
:101DC00058078FEF68078FEF780721F4A1E0CA2E3C
:101DD000D12C24C0CB01BA01F3E0660F771F881F16
:101DE000991FFA95D1F7209110023091110240917C
:101DF000120250911302620F731F841F951FA801D6
:101E00009701E4E0220F331F441F551FEA95D1F7D5
:101E10000E94A41469010894C108D10898A99923C3
:101E2000C9F1ECA1FDA180819095892380838FEF7A
:101E3000E8168FEFF8068FEF08078FEF180719F4F1
:101E400021E030E01DC032E0EE0CFF1C001F111F2E
:101E50003A95D1F7609110027091110280911202AF
:101E6000909113026E0D7F1D801F911FEE0CFF1CC1
:101E7000001F111FA80197010E94A4142150304097
:101E80002C153D0538F0ECA1FDA1808198A9892B86
:101E900080836901E8A5F9A5C082EAA5FBA5D082E7
:101EA000BFBEDF91CF911F910F91FF90EF90DF9018
:101EB000CF90BF900895DC019696ED91FC91979795
:101EC000808187728083D0969C91D097992341F02E
:101ED0009496ED91FC9195978081909589238083CC
:101EE0000895DC0155968C915597882371F096964C
:101EF000ED91FC9197978081877B80839696ED91F9
:101F0000FC9197978081806980830895DC019C967D
:101F1000ED91FC919D9760830895DC0155968C911D
:101F20005597882371F09696ED91FC919797808153
:101F30008F7680839696ED91FC9197978081886447
:101F400080830895CF93DF93EC010E947E0E8D89EC
:101F5000882311F020E90CC08D859E85892B11F016
:101F600020E901C020E08F859889892B09F0286439
:101F7000EEA1FFA12083DF91CF910895DC01262FF0
:101F800014968D919C911597892B59F01496ED918B
:101F9000FC91159716966D917C911797822F099554
:101FA00008959096ED91FC919197CD010995089532
:101FB000FC0122A133A1F90109950895DF93CF9384
:101FC0000F92CDB7DEB7FC0180819181BE016F5FBA
:101FD0007F4F0E941111882319F42FEF3FEF03C0A8
:101FE0008981282F30E0C9010F90CF91DF910895AA
:101FF000CF93DF93EC01888199810E945911882346
:1020000031F488858460888785EF0E949F0CDF917A
:10201000CF910895FC014FB7F894238534858FEF55
:102020009FEF948783874FBFC9010895FC01838583
:1020300094858F5F9F4F29F4862F90E09487838744
:10204000089580858460808785EF0E949F0C0895A5
:10205000DC0119968D919C911A970296FC012591AD
:102060003491CD01F90109950895CF93DF93EC01E7
:1020700088858E7F8887EE89FF89309721F0888D4B
:10208000998D6FEF0995E985FA85389625913491F8
:102090002115310519F0CE01F9010995DF91CF9194
:1020A0000895CF93DF93EC01888581608887E98567
:1020B000FA853A96259134912115310519F0CE0112
:1020C000F9010995EE89FF89309721F0888D998D66
:1020D00060E00995DF91CF910895EF92FF920F9301
:1020E0001F93CF93DF938C017B01EA010BC0D701D3
:1020F0006D917D01D8015C96ED91FC915D97C801D1
:1021000009952197209799F7DF91CF911F910F9112
:10211000FF90EF9008951F93FC01162F248D358DAD
:10212000F9010995812F1F910895FC01268D378DA6
:10213000F90109950895FF920F931F93DF93CF93B1
:102140000F92CDB7DEB78C01FFB6F894FC01828107
:102150009381BE016F5F7F4F0E941111882329F088
:10216000C80169810E94281007C0C8010E9451104F
:10217000F80180858D7F8087FFBE0F90CF91DF9122
:102180001F910F91FF9008950F931F93CF93DF93AB
:10219000162FEC0102C00E94CA118A819B810E9405
:1021A00051118823C1F70FB7F894888581FD0BC0C2
:1021B000888582608887CE010E943510CE01612F0C
:1021C0000E94281005C08A819B81612F0E945911AD
:1021D0000FBFDF91CF911F910F9108951F931FB7EC
:1021E000F8940E9451101FBF1F9108950F931F93E1
:1021F000CF93DF93062FEC0102C00E94CA1188859D
:1022000080FFFBCF1FB7F894CE010E943510CE019E
:10221000602F0E9428101FBFDF91CF911F910F9157
:102220000895CF93DF93DC01EB014FB7F89400974B
:1022300099F112968D919C911397892B69F11496BF
:102240008D919C911597892B39F116962D913C9182
:102250001797ED91FC911197E20FF31F808188830E
:102260002F5F3F4F17963C932E93169712968D91A2
:102270009C9113972817390721F417961C921E92E8
:10228000169714968D919C911597019715969C938E
:102290008E9314978FEF01C080E04FBFDF91CF91F5
:1022A00008950E941012892B11F080E008958FEF9D
:1022B00008951F93CF93DF93EC01462F1FB7F89437
:1022C0002C813D816A817B812617370710F080E0E1
:1022D00011C08E819F81820F931F0E949014E8810C
:1022E000F981E80FF91F40838C819D8101969D83C0
:1022F0008C838FEF1FBFDF91CF911F9108950F93B4
:102300001F9300E010E00E9488111F910F91089523
:102310008F929F92AF92BF92CF92DF92EF92FF92F5
:102320000F931F93CF93DF936B017C0149015A01F7
:10233000E8010E94E30B6C197D098E099F0968155D
:1023400079058A059B0568F00115110541F06819AA
:1023500079098A099B09688379838A839B838FEF34
:102360000CC00115110541F0861A970AA80AB90A8E
:1023700088829982AA82BB8280E0DF91CF911F91EF
:102380000F91FF90EF90DF90CF90BF90AF909F9014
:102390008F9008958FB7789400000000000000002F
:1023A0000000000000008FBF0895662319F00E940E
:1023B000461208950E9421120895613023E07207A9
:1023C00020E0820720E0920748F423E030E040E07C
:1023D00050E00E94A4142A95F1F708959B01AC01E6
:1023E00082E056954795379527958A95D1F7DA017A
:1023F000C901203060E0360761E0460760E056071B
:1024000020F08FEF9FEFA0E0B0E0FC013197F1F7F3
:10241000A0E0B0E0281B390B4A0B5B0B41F7089595
:10242000FC014FB7F894009719F420E030E006C0A3
:102430002281338184819581281B390B4FBFC901CB
:102440000895CF93DF939C010097E9F0FC018591FB
:102450009491FC01A591B4910296FC01C591D4918F
:102460002E5F3F4FF90124918881822349F09FB765
:10247000F8948C91209582238C939FBF000003C019
:1024800087EF0E949F0CDF91CF910895CF93DF9348
:102490009C010097E1F0FC0185919491FC01A591CC
:1024A000B4910296FC01C591D4912E5F3F4FF90182
:1024B00024918881822341F09FB7F8948C91822BDC
:1024C0008C939FBF000003C087EF0E949F0CDF9199
:1024D000CF9108956F927F928F929F92AF92BF9209
:1024E000CF92DF92EF92FF920F931F93DF93CF93E0
:1024F000CDB7DEB72B970FB6F894DEBF0FBECDBFBA
:102500005C014B017A01FC0117821682838181FDF7
:1025100008C06FEF7FEF08C142E050E0E40EF51E07
:1025200004C03E010894611C711CF501D380F401C4
:10253000D3FC8591D3FE81914F01882309F4F1C02A
:10254000853259F4D3FC6591D3FE61914F01653218
:1025500019F0062F10E01BC085E290E02BC000238D
:1025600009F4DFC087E291E0602F70E00E94AD13B4
:10257000892B39F4033211F4106103C00C3661F475
:102580001068F401D3FC0591D3FE01914F0117FFB0
:10259000E6CF002309F4C5C080E291E0602F70E02F
:1025A0000E94AD13892B51F044E050E0E40EF51E7B
:1025B0008FE390E0B5010E94D613B7CF033629F020
:1025C000033779F00335F1F40BC087010E5F1F4F1D
:1025D000F70180819181B5010E94D6137801A5CFC2
:1025E0001160F701C080D18004C090E0B5010E9465
:1025F000D613F60110FD859110FF81916F0188239C
:10260000A1F78ACF043611F0093639F517FF08C053
:10261000F701208131814281538184E090E00AC03A
:10262000F701808191819C01442737FD4095542F0B
:1026300082E090E0E80EF91E1F7E57FF08C050951B
:102640004095309521953F4F4F4F5F4F1064CA0121
:10265000B901A3012AE030E034C00037A9F0013706
:1026600030F40835B1F00F3609F05BC006C005370D
:1026700039F0083709F055C008C028E030E00CC038
:102680001F7E2AE030E008C01061146220E130E0D3
:1026900003C0146020E132E017FF08C0F701608139
:1026A00071818281938144E050E008C0F70180810C
:1026B0009181BC0180E090E042E050E0E40EF51E24
:1026C000A3010E941314D82ED618012F10E006FF84
:1026D00005C08DE290E0B5010E94D61304FF15C03D
:1026E000FE01ED0DF11D8081803379F080E390E0F3
:1026F000B5010E94D61302FF08C000721070C80115
:10270000885A9F4FB5010E94D613DA94F301ED0D5C
:10271000F11D808190E0B5010E94D613DD20A9F75C
:1027200004CFF50166817781CB012B960FB6F89423
:10273000DEBF0FBECDBFCF91DF911F910F91FF90F4
:10274000EF90DF90CF90BF90AF909F908F907F9051
:102750006F900895F8940C94C614FC010590061629
:1027600021F00020D9F7C00108953197CF010895D5
:102770000F931F93DF93CF93CDB7DEB70F811885EB
:102780009E01255F3F4FF801838188608383C801E4
:1027900069857A85A9010E946A12F8012381277F41
:1027A0002383CF91DF911F910F9108950F931F9372
:1027B000CF93DF938C01EB018B8181FF1BC082FFE4
:1027C0000DC02E813F818C819D812817390764F4CB
:1027D000E881F9810193F983E88306C0E885F985EA
:1027E000802F0995892B31F48E819F8101969F83DB
:1027F0008E8302C00FEF1FEFC801DF91CF911F91B1
:102800000F9108950F931F938C01FC0183818860C1
:102810008383C8010E946A12F8012381277F2383E2
:102820001F910F910895FA01AA27283051F1203104
:1028300081F1E8946F936E7F6E5F7F4F8F4F9F4F54
:10284000AF4FB1E03ED0B4E03CD0670F781F891F96
:102850009A1FA11D680F791F8A1F911DA11D6A0F64
:10286000711D811D911DA11D20D009F468943F9117
:102870002AE0269F11243019305D3193DEF6CF0116
:102880000895462F4770405D4193B3E00FD0C9F7DC
:10289000F6CF462F4F70405D4A3318F0495D31FD49
:1028A0004052419302D0A9F7EACFB4E0A69597959C
:1028B000879577956795BA95C9F700976105710572
:1028C00008959B01AC010A2E0694579547953795BC
:1028D0002795BA95C9F7620F731F841F951FA01D16
:1028E0000895629FD001739FF001829FE00DF11D5A
:1028F000649FE00DF11D929FF00D839FF00D749F7A
:10290000F00D659FF00D9927729FB00DE11DF91F25
:10291000639FB00DE11DF91FBD01CF011124089582
:10292000AA1BBB1B51E107C0AA1FBB1FA617B707F5
:1029300010F0A61BB70B881F991F5A95A9F7809511
:102940009095BC01CD010895A1E21A2EAA1BBB1BD4
:10295000FD010DC0AA1FBB1FEE1FFF1FA217B3076B
:10296000E407F50720F0A21BB30BE40BF50B661F81
:10297000771F881F991F1A9469F760957095809545
:1029800090959B01AC01BD01CF010895F894FFCF54
:102990000A1168656C6C6F20776F726C6421000699
:1029A0000024F400803E1000AE02BA0200000000D5
:1029B000009406FFFF1F0422047A0B860B00000020
:1029C00000000000C4109B10F80FDE0FC000C10013
:1029D000C400C500C60000000200000000000000A6
:1029E00000009406FFFF16041904750B7F0B00000E
:1029F0000000000000F610EE1016100A10C800C902
:102A000000CC00CD00CE00000002083404002504F4
:102A1000310437040000000200000000FE0900003D
:102A200000000000000200000000FE09000000009D
:102A3000000000010000000000000B0A000060031D
:102A400050000000000000000000B0035000000033
:102A50000000000000001E0E000000020000000048
:062A6000600E430E0000B1
:00000001FF
